:1052B600AB38AA39A93A854282758300123516FFA2
:0452C600AC40AD410A
:1052CA00AB07C2AF75F65575F6AA75F65543BF0416
:0F52DA008CF4EDF5F58BF675F780D2AF7F0022DF
:10550300C2AFE4FEEEC39D501B75F65575F6AA7542
:10551300F65543BF04EF25E0F5F4E4F5F575F7829E
:065523000F0E80E0D2AF84
:01552900225F
:0B5670008F828E83E4931235437F018C
:01567B00220C
:0C552A00E52F75F002A42408F9E4FAFB58
:10553600123614F58285F083E4932402FFE4338F58
:04554600F002363FFA
:10531C008D3EA907E925E02408F8E6FE08E6FFED36
:10532C002402FDE433FCE925E02471F8E6FA08E6F2
:10533C00C39DFDEA9CFCD3EF9DEE9C4002D322C39F
:01534C00223E
:062EC3008F2F8D308B31D2
:102EC900E53025E0F534753500E53125E07536FF47
:102ED900F537753800853582853483E49364556008
:102EE9000302303BAB36AA37A9381234FD6455606A
:102EF9000302303BE5352401FFE43534FEE52F2597
:102F0900E02408F8A60608A607E52F25E02408F816
:102F1900E6FE08E6F5828E83E493F46020E52F252A
:102F2900E02408F8E6FE08E6AA06C3853783853853
:102F3900829582EA9583500512552A80CCE52F2582
:102F4900E02408F8E6FE08E6C39535FFEE9534F56A
:102F5900398F3AE5382401F9E43537FEAF01E52F19
:102F690025E02408F8A60608A607E52F25E0240889
:102F7900F8E6FE08E6F5828E83E493F46030AB361A
:102F8900E5382533F9E5373532FAC0038A83898272
:102F9900E52F25E02408F8E6FE08E6AA06F9C3D0DD
:102FA900E0E99582EA9583500512552A80BCE52F00
:102FB90025E02408F8E6FE08E6AB36AA37A938ACBE
:102FC90002AD01C39DFFEE9CFED3EF953AEE953914
:102FD9005033AE02AF01EF2401FFE43EFEE52F2599
:102FE900E02463F8A60608A607747B252FF8A63007
:102FF900AE34AF35AD07AC06E4FF1252CAEF700329
:103009000230BCC322E5352401FFE43534FEE52F47
:1030190025E02463F8A60608A607747B252FF8A6E1
:1030290031AC37AD38E4FF1252CAEF70030230BC3D
:10303900C322853582853483E493B4551EE535244E
:1030490001FFE43534FEE52F25E02463F8A60608E0
:10305900A607747B252FF8A6318058AB36AA37A965
:10306900381234FDB45520AE02AF01EF2401FFE45C
:103079003EFEE52F25E02463F8A60608A607747B23
:10308900252FF8A630802CAE34AF35AD07AC06ED50
:103099002401FFE43CFEE52F25E02463F8A6060899
:1030A900A607747B252FF8A6317F551252CAEF6007
:1030B90002C322E52F25E02463F8E6FE08E6FFE5D2
:1030C9002F25E02408F8A60608A607E52F25E02401
:1030D90064F8E62533FF18E63532FEE52F25E024AE
:1030E90071F8A60608A607E52F25E02408F8E6FEEC
:1030F90008E6F5828E83E493F4600512552A80E789
:01310900D3F2
:01310A0022A2
:063BE8008F3E8C3F8D4072
:103BEE00EF25E02463F8E6FE08E68E41F542747B8D
:103BFE002FF8E625E0F545754600E5422540FFE540
:103C0E0041353FCF24FFF544EF34FFF543E53FC385
:103C1E0013F5471254AF747B253EF8E6FFAD4712FD
:103C2E0055030546E546700205458542828541836A
:103C3E00E493F47003023D04C3E5429544E54195D7
:103C4E00434003023D041254AF8542828541837482
:103C5E000193FF7003023CF8F47003023CF8054236
:103C6E00E542AE417002054114F5828E83E493F570
:103C7E0048AE45AF46AD07AC06FF1252CAEF600321
:103C8E007F01220546E546700205450542E542AE36
:103C9E00417002054114F5828E83E493FFAC45AD6D
:103CAE00461252CAEF60037F01220546E5467002B6
:103CBE000545E4F547E547C395484003023C380502
:103CCE0042E542AE417002054114F5828E83E493C3
:103CDE00FFAC45AD461252CAEF60037F0122054686
:103CEE00E54670020545054780CB7B007A00794199
:103CFE00125536023C38E53E25E02408F8A6450864
:103D0E00A646E53E25E02463F9E7C313FD747B2543
:103D1E003EF8E625E0FEE53E25E02463F8A606081B
:103D2E007600747B253EF8A605E53E25E02464F872
:103D3E00E62540FF18E6353FFEE53E25E02471F806
:103D4E00A60608A607E53E25E02463F8E6FC08E68D
:103D5E00FD7F551252CAEF60037F0122747B253E10
:103D6E00F8E67F0025E0FE7D00FC1252CAEF6003EC
:103D7E007F0122E53E25E02463F80806E61870016F
:033D8E00067F00AD
:013D9100220F
:083D92008F3E8B3F8A408941FE
:103D9A00E4F547F548E54325E02463F8E6FE08E63E
:103DAA008E44F545053EE54325E02408F8E6FE087D
:103DBA00E6FFE5422401FDE433FCE54325E02472F5
:103DCA00F8C3E69DFD18E69CFCD3EF9DEE9C4001EE
:103DDA0022854582854483740193FE653E6010E422
:103DEA0093F4600B7B007A00794412553680E2EE38
:103DFA00B53E0BE5452401F548E43544F547E5436E
:103E0A0025E02408F8E6FE08E6FDAC06AF421252A9
:103E1A00CAEF6002C322E54325E02408F8087402C9
:103E2A0026F618E436F6E54364047023E54325E0F4
:103E3A002408F8E6FE08E6FDAC06AB3FAA40A94115
:103E4A001234FDFF1252CAEF7003023ED7C322E4B6
:103E5A00F546E546C395425074AB3FAA40A9419046
:103E6A00FFFE123516FE90FFFF1235166E7026E51C
:103E7A004325E02408F8E6FE08E62546FFE43EFE70
:103E8A00AD07FC854682758300123516FF1252CAA9
:103E9A00EF6036C322E54325E02408F8E6FE08E68B
:103EAA002546FFE43EAD07FCE54625E0FFE433FE88
:103EBA00AB3FE5412FF9E5403EFA90000112351675
:103ECA00FF1252CAEF6002C32205468085AF427EC6
:103EDA0000E54325E02408F808EF26F618EE36F642
:103EEA00E54325E02408F8E6FC08E6FDEF2401FF97
:103EFA00EE33FEC3ED9FFFEC9EFEAD07FCAF3E1214
:103F0A0052CAEF6002C322E54845476012AE47AF86
:103F1A0048AD07AC06E4FF1252CAEF6002C322D3CF
:013F2A002274
:044AF0008F358D363B
:104AF400E53625E02463F8E6FE08E68E37F538E46B
:104B0400F539F53A0535853882853783E493F460C1
:104B14004BE53625E02471F8E6FC08E6FDC3E538EC
:104B24009DE5379C503674019365357024E53A450C
:104B3400396018E53A2401FFE43539FEAD07FCE499
:104B4400FF1252CAEF6004E4FEFF2285373985382C
:104B54003A7B007A00793712553680AAE53A45390E
:104B6400600AE53A2402FFE43539FE227EB47FDC94
:014B7400221E
:0851D1008F358B368A378938CF
:1051D900E4F53D1254AFAD39AF3A12531C500EAD40
:1051E9003CAC3BAF3A123BE8EF6002053DE53D7050
:1051F90011AB36AA37A938853942853A43AF3512FA
:035209003D92D300
:01520C00227F
:0446F4008F2F8D3047
:1046F800EF25E0F531753200E4F533F534E534C3E0
:104708009530501EE5347F0025E0FEEF2532F58216
:10471800E5313EF583E493D394084002053305342C
:1047280080DB7D047F09124AF08F828E83E493B484
:104738008807E533D3940140307533887B007A00CD
:104748007933753901753A04753B02753C007F0968
:104758001251D1E4F533E52F2533FF7D01125503BE
:104768000533E533C3940840EDE52F25E0F53175B1
:104778003200853282F583E493F4703E2582F58217
:10478800E5833402F583E493F4702FF533E53014B0
:10479800FFE533C39F5019E53325E0FEE42532FFDA
:1047A800EE3531FEAD07FCAF331252CA053380DD5A
:1047B800E52F2530147880F6D322E4F534E534C3A8
:1047C8009530502BE5347F0025E0FEEF2532F58249
:1047D800E5313EF583E493D39408400FE52F253463
:1047E800FF7880F67D01125503D322053480CED39D
:0147F800229E
:065248008D44AC07A90330
:10524E00EC25E07B00FAE4FDEDC395465020ED7FA2
:10525E000025E0FEEF2BF582EA3EF583E493FFE5B1
:10526E004489F084B50704EC2DFF220D80DAAF04DB
:01527E00220D
:063F2B008D358B36AC075A
:103F3100E4F5427880E67F0025E0FE786FF608EF31
:103F4100F62402FFE43EF5408F41AF04853746ABCE
:103F510036AD351252487880EFF67F0025E0FE78C5
:103F61006DF608EFF62402FFE43EF53E8F3F125452
:103F7100AFE4F53CE5358536F084E53CC395F0507A
:103F810034E4F53DE53DC3953B5026053FE53FAEA5
:103F91003E7002053E14F5828E83E4931252C5EF02
:103FA10060037F01220541E54170020540053D8026
:103FB100D3053C80BFE4F53DE53BC313FFE53DC3BD
:103FC1009F4003024067E53D30E003024057AB38B4
:103FD100AA39A93A90FFFE123516FF90FFFF12355C
:103FE100166F604AE54275F002A429F9EA35F0FA44
:103FF1009000011252C2EF60037F01220541E541A9
:10400100700205400542E54275F002A4AB38253A3D
:10401100F9E53935F0FA9000011252C2EF60037FE1
:1040210001220541E54170020540054280331252EB
:10403100B6EF60037F01220541E5417002054005AD
:10404100421252B6EF60037F01220541E541700241
:1040510005400542800B74022541F541E43540F5E8
:1040610040053D023FB9E53B253FF53FE4353EF5CF
:104071003EE5358536F084E5F004F53CE53CC39535
:10408100365034E4F53DE53DC3953B5026053FE50B
:104091003FAE3E7002053E14F5828E83E4931252C8
:1040A100C5EF60037F01220541E54170020540052E
:0740B1003D80D3053C80C5F2
:0140B80022E5
:0644AC008B368A378938C7
:1044B200E4F53D786FE6FA08E68A3AF53BEF8DF0CF
:1044C20084E5F0FD7C00AF397E00123577EF2404DD
:1044D200FFE43EFEEF253BF53BEE353AF53AE4F5D7
:1044E2003CE539C313FFE53CC39F40030245C9E5E0
:1044F2003C30E0030245B9AB36AA37A93890FFFE3B
:10450200123516FF90FFFF1235166F605AE53D75A2
:10451200F002A429F9EA35F0FA900001123516FFEB
:10452200AC3AAD3B1252CAEF60037F0122053BE574
:104532003B7002053A053DE53D75F002A4AB362518
:1045420038F9E53735F0FA900001123516FFAC3A2A
:10455200AD3B1252CAEF60037F0122053BE53B707F
:1045620002053A053D805BAB36AA37A938853D8204
:10457200758300123516FFAC3AAD3B1252CAEF609A
:10458200037F0122053BE53B7002053A053DAB3650
:10459200AA37A938853D82758300123516FFAC3AD9
:1045A200AD3B1252CAEF60037F0122053BE53B702F
:1045B20002053A053D800B7402253BF53BE4353A92
:1045C200F53A053C0244E3786DE6FE08E6F5828E94
:1045D20083E493FF08E6FC08E6FD1252CA7880E6FF
:0645E200FF7D01125503EC
:0145E80022B0
:0453DC008D368B3748
:1053E000853846125248EF25E07D00FCED2402FD91
:1053F000E43CFCE5368537F084E5F075F090A42DAB
:07540000FDE5F03CFEAF05E5
:015407002282
:0300030002567C26
:0C567C00D2D8C2D9756201D25EC25F3282
:030013000256880A
:0C568800D2D8D2D9756201D25FC25E3266
:05520D000320FFFFFF7C
:104A6800781DE675F00384E5F014600D14601D24CC
:104A7800027074852080D2B722E54EC3940C50048E
:104A8800054E8002D20E852180D2B622E54AC39413
:104A98000C500E054AE54AB40A10C216E4F54C80DB
:104AA80009304504D2158002D216E54BC3940C5048
:104AB8000E054BE54BB40A10C213E4F54D800930DE
:104AC8004704D2128002D213E54CC3940C5004055B
:104AD8004C8002D216E54DC3940C5004054D80025B
:084AE800D213852280D2B52211
:03000B000254B3E9
:1054B300C0E0C0F0C0D075D000C000781D06758A6A
:1054C30000758CEED253C2B7C2B6C2B5124A68D0C9
:0854D30000D0D0D0F0D0E0328F
:1055FD00001E000A0014012C00C8006400C81644E7
:02560D0004880F
:09521200012300C152C155C15431
:10548A007F507EC31256941254AF7F507EC3125679
:10549A00941254AF7F507EC31256941254AF7F5069
:0554AA007EC3125694C0
:0454AF00759FA6221D
:0C569400EF4E6007EF1F70F81E80F5223B
:10527F00AB07ED7015EB25E024FDF582E43455F511
:10528F0083E493FE740193FF800BAF057E007C00D7
:10529F007D0A123577EB25E0246AF582E43402F5B6
:0752AF0083EEF0A3EFF022F3
:10560F00EF25E0246AF582E43402F583E4F0A3F099
:01561F002268
:0A56A0007F1290026AE4F0A3DFFC21
:0156AA0022DD
:1022FB0090027D74C8F09002927406F0E4A3F09003
:10230B00029DF0D2A7900269F09000D3F0754A328B
:10231B00754B321256A07B007A00798B7D01E4FF5E
:10232B00124D9F788BE66006E4FDFF12554AE49050
:10233B000001F0A3F0900031F0A3F07887F608F6D7
:10234B009001D4F0900030F0900000F0753204F55D
:10235B00337B5D7D5BFF122EC37532047533007BBF
:10236B00617D5F7F01122EC37532067533007B666C
:10237B007D637F02122EC37532047533007B6B7D38
:10238B00697F03122EC37532027533007B767D7520
:10239B007F04122EC37D087F6D1246F4E4FD7F0788
:1023AB0012527FE4FD7F0212527FE4FD7F03125233
:1023BB007F7D287F0412527FE490023FF0A374B814
:1023CB00F0E4A3F0788BF6788BE6FFC39427500FDD
:1023DB0074092FF582E43400F583E4F00680E8E419
:1023EB00788BF6788BE6FFC394205033741B2FF554
:1023FB0082E43402F583E4F074D52FF582E43401E2
:10240B00F583E4F074F52FF582E43401F583E4F001
:10241B0074482FF582E43402F583E4F00680C4E4BB
:10242B00788BF6788BE6FFC39403502774452FF512
:10243B0082E43402F583E4F074152FF582E4340260
:10244B00F583E4F074182FF582E43402F583E4F09D
:10245B000680D0E4788BF6788BE6FFC39402500F9E
:10246B00743B2FF582E43402F583E4F00680E81226
:10247B0054AFE4788BF6788BE6FFC394FF500F7460
:10248B00D52FF582E43400F583E4F00680E8E47898
:10249B008BF6788BE6FFC394A0500F74332FF58225
:1024AB00E43400F583E4F00680E87B007A00795E83
:1024BB007F067EEF125670E55EF46004E55E7011E8
:1024CB007D047F06124AF08F828E83E493F55E8043
:1024DB00177B007A00795E753901753A04753B02FA
:1024EB00753C007F061251D1E55E6003B4FF0375A6
:1024FB005EFE7D047F63124AF08F828E83E493F538
:10250B005DD394084067E4F55DFB7A00795D75391E
:10251B0001753A04753B02F53C7F631251D1788B00
:10252B0076677B007A00798B753901753A04753BB8
:10253B0002753C007F041251D1E4788BF6FB7A00D4
:10254B00798B753901753A04753B02F53C7F0512A1
:10255B0051D1788B76647B007A00798B7539017554
:10256B003A04753B02753C007F071251D17D047F05
:10257B000E124AF08F828E83E49390027CF0E0D3AC
:10258B0094024038E4900268F07B017A0279687516
:10259B003901753A04753B02F53C7F0D1251D1E4BC
:1025AB0090027CF07B017A02797C753901753A04D3
:1025BB00753B02F53C7F0E1251D180117D047F0DCE
:1025CB00124AF08F828E83E493900268F0759850D4
:1025DB0075891175CDFF75CCB875CBFF75CAB8D29F
:1025EB00CDD2CCC2CBC2C9C2C8D2CAE4F58DF58B51
:1025FB00F58A758CEEC28ED28CD2A9D288D2A8D293
:10260B008AD2AAD2AFD2ACD2BC7D047F0C124AF0D4
:10261B008F828E83E493788BF6E6B40118900029B1
:10262B007401F0C2CA75CDFF75CCDC75CBFF75CAD2
:10263B00DCD2CA8015E4900029F0C2CA75CDFF75B3
:10264B00CCB875CBFF75CAB8D2CA78897601124D52
:04265B0043755CA1C6
:01265F002258
:1055C400D25F1254AFC25E125582759955C24430EF
:0355D40044FD2271
:104E5100D25F1254AFC25E12558290027DE0F59985
:104E6100C2443044FD855E99C2443044FDE4FF7480
:104E7100092FF582E43400F583E0F599C24430440A
:104E8100FD0FBF06EA900292E0F599C2443044FD5D
:104E9100900293E0F599C2443044FD90029DE0F503
:064EA10099C2443044FDFB
:014EA70022E8
:104B7500EFB40900507B904B82F8282873024B9DB7
:104B8500024BA4024BA7024BB7024BC4024BD10206
:104B95004BDD024BE4024BECC218D2AAD2A822C2CA
:104BA5001922122660E5237003122C40E4FD7F02D2
:104BB500803CE52370031245E9E4FD7F03802FE582
:104BC50023700312330BE4FD7F048022124F8BD236
:104BD500A7E5152464F51522D214D217D20F22D2D7
:104BE50055E4FD7F078007124E51E4FD7F08125200
:024BF5007F221D
:1036C900C249D292D2A012548AC292C2A012548A7A
:1036D9001222FB7D047F05124AF08F828E83E493C8
:1036E900752C00F52D7D047F04124AF08F828E839C
:1036F900E493FD7C00E52DFEE42DF52DEC3EF52C43
:10370900E52D6415452C6032E4F52EFB7A00792EFF
:10371900753901753A04753B02F53C7F051251D1A3
:10372900752E157B007A00792E753901753A047565
:103739003B02753C007F041251D120530302381C0F
:10374900305B0E20490BC25BD2497D057F081252BE
:103759007F305D05C25D1255C4D3900032E09400FC
:10376900900031E094004022A3E024FFF090003162
:10377900E034FFF0E07002A3E0700FD2AAD2A8F5FE
:1037890062788AF69000D3F0C218D3900002E094D0
:1037990000900001E09400402BA3E024FFF090008A
:1037A90001E034FFF0E07002A3E0701830520ED24D
:1037B900D8C25285496190003004F08005E4F5498A
:1037C900C219D20DD37888E6940018E694004020F7
:1037D90008E616187001167888E6184670129000E7
:1037E90000E0B40103854961900000E004F0D25C77
:1037F900C253900030E060031256429001D4E06059
:10380900031248F6900000E0D394004006305C03B0
:10381900120E12781DE6D394275003023743E4F6BB
:10382900900269E004F0E0B40804E4F0B211125423
:10383900AFE4F51CE51CC394094003023743E51CBA
:1038490025E0246AF582E43402F583E0FEA3E0FF73
:10385900781EEEF608EFF64E6027E6161870011688
:10386900781EE6FE08E6FFE51C25E0246AF582E4F9
:103879003402F583EEF0A3EFF04E7005AF1C124B46
:0538890075051C80AF75
:10310B0000C1814001C0804101C0804100C18140AC
:10311B0001C0804100C1814000C1814001C080419C
:10312B0001C0804100C1814000C1814001C080418C
:10313B0000C1814001C0804101C0804100C181407C
:10314B0001C0804100C1814000C1814001C080416C
:10315B0000C1814001C0804101C0804100C181405C
:10316B0000C1814001C0804101C0804100C181404C
:10317B0001C0804100C1814000C1814001C080413C
:10318B0001C0804100C1814000C1814001C080412C
:10319B0000C1814001C0804101C0804100C181401C
:1031AB0000C1814001C0804101C0804100C181400C
:1031BB0001C0804100C1814000C1814001C08041FC
:1031CB0000C1814001C0804101C0804100C18140EC
:1031DB0001C0804100C1814000C1814001C08041DC
:1031EB0001C0804100C1814000C1814001C08041CC
:1031FB0000C1814001C0804101C0804100C18140BC
:10320B0000C0C101C30302C2C60607C705C5C4047B
:10321B00CC0C0DCD0FCFCE0E0ACACB0BC90908C8EB
:10322B00D81819D91BDBDA1A1EDEDF1FDD1D1CDCDB
:10323B0014D4D515D71716D6D21213D311D1D0104B
:10324B00F03031F133F3F23236F6F737F53534F43B
:10325B003CFCFD3DFF3F3EFEFA3A3BFB39F9F838AB
:10326B0028E8E929EB2B2AEAEE2E2FEF2DEDEC2C9B
:10327B00E42425E527E7E62622E2E323E12120E00B
:10328B00A06061A163A3A26266A6A767A56564A4FB
:10329B006CACAD6DAF6F6EAEAA6A6BAB69A9A8686B
:1032AB0078B8B979BB7B7ABABE7E7FBF7DBDBC7C5B
:1032BB00B47475B577B7B67672B2B373B17170B0CB
:1032CB0050909151935352929656579755959454BB
:1032DB009C5C5D9D5F9F9E5E5A9A9B5B995958982B
:1032EB00884849894B8B8A4A4E8E8F4F8D4D4C8C1B
:1032FB00448485458747468682424383418180408B
:10521B00018A004100D300014900C144C143C1C010
:02522B00C1467A
:10559900C2B4756203E4F549900030F0C2D8D2D99B
:0655A9007F0AFE02569489
:1055D700C20EE4F54ED244D2B4C2A3D2A47F0AFECF
:0355E700025694D5
:10558200E4F562C244305E05D2A3C2A422305F06B3
:07559200D2A3D2A4D295229E
:0756B600755BFF755AFF222E
:07556700853399C244AF3304
:10556E00E55A6FFF90310B93655BF55AEF90320B56
:03557E0093F55B47
:015581002207
:08501A008B3B8A3C893D8D3E71
:10502200753F007540FF7DFFAF3E153EEF6026AB3A
:105032003B053DE53DAA3C7002053C14F91234FDE6
:105042006540FF90310B936D753F00F540EF903254
:0A5052000B93FD80D3E540FEEDFF57
:01505C002231
:084EF5008B368A378938AC05C1
:104EFD00EC24FEFD12501A8E398F3AEC7E0024FE02
:104F0D00F582EE34FFF583AB36AA37A93812351684
:104F1D00FEAD047C0074FF2DF582EC34FFF5831299
:104F2D0035162400FFEC3EFEEFB53A06EEB539021C
:034F3D00D322C3B9
:014F4000224E
:10388E00900033E0FFF4600AEF655E6005EF6002C2
:10389E00C322900034E0641A6003023937205F2A95
:1038AE007B017A0079337D0412501A8E2F8F30905F
:1038BE000037E0FEA3E07C002400FFEC3EFEEF6547
:1038CE00307003EE652F6002C322900036E0FF9049
:1038DE000035E0FEC39F40028002AF06900036E046
:1038EE00FDEEC39D4007900035E0FE8002AE05E57B
:1038FE005EC39F4006E55ED39E4002C322781DE65E
:10390E00FF7E00124EEA124EA87C007D0A1235DEB2
:10391E008D31E4F532E532C39531500B7F4B7E008D
:10392E00125694053280EED322900034E0FF6403E9
:10393E00600CEF64066007EF64106002C322900013
:10394E0035E0FEA3E07C002400FFEC3EFEEF640AAF
:10395E004E704E900034E0B4031C124EA87C007DD5
:10396E000A1235DE7E007F02CFCDCFCECCCE123501
:10397E00DE9000D4EFF09000D4E064016002C32228
:10398E00124EA87C007D0A1235DE8D31E4F532E54B
:10399E0032C39531500B7F4B7E0012569405328008
:1039AE00EE900034E064067042A3E0FEA3E07C00DB
:1039BE002400FFEC3EFEC3EF9404EE64809480403E
:1039CE000CEF64084E6006EF64074E701E900036D2
:1039DE00E0FFC394025007E55D30E00FC322EFC352
:1039EE0094045007E55D30E102C322305F02D3221A
:1039FE007B017A007933E55024FEFD12501A8E2F8A
:103A0E008F3074312550F582E43400F583E0FE7476
:103A1E00322550F582E43400F583E07C002400FF6B
:0E3A2E00EC3EFEEFB53006EEB52F02D322D3EC
:013A3C002267
:08537E008F368B378A3889391C
:10538600E4FF1255D7E4FFEFC395365018AB37AAA2
:1053960038A9398F82758300123516F599C24430C3
:0853A60044FD0F80E20255995D
:10534D00E49002A2F09002A2E0FEC39405501A74FC
:10535D00032EF582E43400F583E0F599C244304420
:10536D00FD9002A2E004F080DC8F99C2443044FD30
:01537D00220D
:10028C00E4F532900034E0FD64067034305F0A7F90
:10029C000612534D7531068003753108E4F532E5CD
:1002AC0032C395314003020E1174332532F582E4CA
:1002BC003400F583E0F599C2443044FD053280DF0B
:1002CC00ED64036003020D6F900035E0FEA3E07C4B
:1002DC00002400F530EC3EF52F900038E0F531307D
:1002EC005F08E5312403FF12534D900033E0F533E2
:1002FC00125567900034E0F5333044FD125567E534
:10030C003125E0F5333044FD125567E532C39531A4
:10031C004003020D517E00E5302532FFEE352FFEF5
:10032C00D3EF940DEE94005021E4F5333044FD12DC
:10033C005567E5322530FF7D04124AF08F828E839B
:10034C00E493F5333044FD020D497E00E53025324F
:10035C00FFEE352FFEEF64104E701DF5333044FD6B
:10036C001255677D047F10124AF08F828E83E493BE
:10037C00F5333044FD020D497E00E5302532FFEEA9
:10038C00352FFEEF640F4E701DF5333044FD1255C2
:10039C00677D047F0F124AF08F828E83E493F533CE
:1003AC003044FD020D497E00E5302532FDEE352F3F
:1003BC00FCED645A4C7011F5333044FD12556785D1
:1003CC0026333044FD020D49ED64634C701DF5334A
:1003DC003044FD1255677D047F63124AF08F828E84
:1003EC0083E493F5333044FD020D497E00E530255E
:1003FC0032FFEE352FFEC3EF9464EE94004027EFEE
:10040C00946AEE9400501FE4F5333044FD125567A6
:10041C00E532253024A5F582E434FFF583E0F5338D
:10042C003044FD020D497E00E5302532FDEE352FBE
:10043C00FCED646A4C7014F5333044FD1255679032
:10044C00000FE0F5333044FD020D49C3ED946BEC25
:10045C00940040337E00E5302532FFEE352FFEC38D
:10046C00EF9477EE9400501FE4F5333044FD1255B1
:10047C0067E532253024A5F582E434FFF583E0F5F9
:10048C00333044FD020D497E00E5302532FDEE355A
:10049C002FFCED64774C7014F5333044FD12556726
:1004AC0090001CE0F5333044FD020D49ED64784CAE
:1004BC00701890001EE0F5333044FD125567900023
:1004CC001DE0F5333044FD020D497E00E530253248
:1004DC00FFEE352FFEC3EF9479EE94004027EF9496
:1004EC007DEE9400501FE4F5333044FD125567E562
:1004FC0032253024A6F582E434FFF583E0F5333061
:10050C0044FD020D497E00E5302532FFEE352FFE0D
:10051C00C3EF947DEE9400403DD3EF947FEE9400B6
:10052C005034E5322530248325E02424F582E4344C
:10053C0000F583E0F5333044FD125567E532253084
:10054C00248325E02423F582E43400F583E0F5339D
:10055C003044FD020D497E00E5302532FDEE352F8D
:10056C00FCED64804C7014F5333044FD12556790EB
:10057C000029E0F5333044FD020D49ED64814C70E7
:10058C001890002BE0F5333044FD12556790002A8B
:10059C00E0F5333044FD020D497E00E5302532FF95
:1005AC00EE352FFEC3EF9482EE94004028D3EF94E7
:1005BC0085EE9400501FE4F5333044FD125567E589
:1005CC0032253024AAF582E434FFF583E0F533308C
:1005DC0044FD020D497E00E5302532FDEE352FFC41
:1005EC00ED64864C7011F5333044FD12556785511E
:1005FC00333044FD020D49ED64874C7011F53330F6
:10060C0044FD1255678552333044FD020D497E007E
:10061C00E5302532FDEE352FFCED64884C7011F57C
:10062C00333044FD1255678553333044FD020D4978
:10063C00ED64894C7011F5333044FD1255678554C7
:10064C00333044FD020D497E00E5302532FDEE3598
:10065C002FFCED648A4C7011F5333044FD12556754
:10066C008555333044FD020D49ED648B4C7011F50A
:10067C00333044FD1255678556333044FD020D4925
:10068C007E00E5302532FDEE352FFCED648C4C7090
:10069C0011F5333044FD1255678557333044FD0254
:1006AC000D49ED648D4C7011F5333044FD125567D6
:1006BC008558333044FD020D497E00E5302532FD6E
:1006CC00EE352FFCED648E4C7011F5333044FD1279
:1006DC0055678559333044FD020D49ED64B94C70B2
:1006EC0014F5333044FD125567900029E0F5333092
:1006FC0044FD020D497E00E5302532FFEE352FFE1C
:10070C00C3EF94C8EE94005003020856EF94D0EE59
:10071C0094004003020856E4F5333044FD1255674B
:10072C007E00E5302532FFEE352FFEEF64C84E70AB
:10073C0020FB7A0079337D017F07124D9F3044FDF9
:10074C00E53330E70675331302085075331402088D
:10075C00507E00E5302532FFEE352FFEEF64C94E9A
:10076C00700FFB7A0079337D017F08124D9F0208D0
:10077C00497E00E5302532FFEE352FFEEF64CA4E80
:10078C007012FB7A0079337D017F07124D9F533332
:10079C001F0208497E00E5302532FFEE352FFEEFB3
:1007AC0064CB4E7012FB7A0079337D017F06124DBB
:1007BC009F5333070208497E00E5302532FFEE35A2
:1007CC002FFEEF64CC4E7011FB7A0079337D017FE4
:1007DC0005124D9F53333F80647E00E5302532FF78
:1007EC00EE352FFEEF64CD4E7011FB7A0079337D20
:1007FC00017F04124D9F53333F80427E00E530252C
:10080C0032FFEE352FFEEF64CE4E7011FB7A00797D
:10081C00337D017F03124D9F53337F80207E00E593
:10082C00302532FFEE352FFEEF64CF4E7016FB7A7B
:10083C000079337D017F02124D9F53337FAF33120A
:10084C0056318F333044FD020D497E00E5302532A0
:10085C00FFEE352FFEC3EF94D0EE94005003020947
:10086C0048EF943CEE94034003020948AF327E00FB
:10087C00E5302532CFEE352FCF2430FBEF34FFFAA5
:10088C007C007D1FAF03FE1235899002A1EFF07C36
:10089C00007D1FAF03AE02123589AF059002A0EFA9
:1008AC00F0700EA3E0FFE4FD124AF08E5F8F6080C3
:1008BC00132041109002A1E0FFE4FD124AF08E5F7C
:1008CC008F60D241E4F5333044FD1255679002A09D
:1008DC00E0FF2560F582E4355FF583E493F533EFB3
:1008EC00641E7052E533F4604DE53320E718900236
:1008FC00A1E0FF7B017A0279451253B650054333D0
:10090C004080035333BF9002A1E0FF7B017A027950
:10091C00151253B6500543332080035333DF900236
:10092C00A1E0FF7B017A0279181253B650054333CC
:10093C001080035333EF3044FD020D497E00E53047
:10094C002532FFEE352FFEC3EF943CEE940350039B
:10095C00020A05EF940CEE94054003020A05AF322F
:10096C007E00E5302532CFEE352FCF24C4FBEF349B
:10097C00FCFA7C007D1DAF03FE1235899002A1EFBD
:10098C00F07C007D1DAF03AE02123589AF059002DD
:10099C00A0EFF0700EA3E0FF7D01124AF08E5F8F86
:1009AC006080132041109002A1E0FF7D01124AF0FB
:1009BC008E5F8F60D241E4F5333044FD1255679061
:1009CC0002A0E0FF2560F582E4355FF583E493F542
:1009DC0033EF641C701DE53320E7189002A1E0FF93
:1009EC007B017A02793B1253B650054333408003A6
:1009FC005333BF3044FD020D497E00E5302532FFF4
:100A0C00EE352FFEC3EF940CEE94055003020AF75B
:100A1C00EF9406EE94084003020AF7AF327E00E52D
:100A2C00302532CFEE352FCF24F4FBEF34FAFA7C9D
:100A3C00007D03AF03FE1235899002A1EFF07C001C
:100A4C007D03AF03AE02123589AF059002A0EFF023
:100A5C00700EA3E0FF7D02124AF08E5F8F60801350
:100A6C002041109002A1E0FF7D02124AF08E5F8FB0
:100A7C0060D241E4F5333044FD1255679002A0E09A
:100A8C00FF2560F582E4355FF583E493F533EF647D
:100A9C00027052E533F4604DE53320E7189002A163
:100AAC00E0FF7B017A02791B1253B65005433340A9
:100ABC0080035333BF9002A1E0FF7B017A0179D50B
:100ACC001253B6500543332080035333DF9002A1F9
:100ADC00E0FF7B017A0179F51253B65005433310D0
:100AEC0080035333EF3044FD020D497E00E5302581
:100AFC0032FFEE352FFEC3EF9406EE94085003023E
:100B0C000BA3EF94E6EE940A4003020BA3EF24FA36
:100B1C00FBEE34F7FA7C007D2EAF03FE123589ED27
:100B2C004C7015FC7D2EAF03AE021235897D03127D
:100B3C004AF08E5F8F608028204125AF327E00E521
:100B4C00302532CFEE352FCF24FACF34F7FE7C0090
:100B5C007D2E1235897D03124AF08E5F8F60D24153
:100B6C00E4F5333044FD125567AF327E00E5302595
:100B7C0032CFEE352FCF24FACF34F7FE7C007D2E0A
:100B8C00123589E5602DF582E55F3CF583E493F53C
:100B9C00333044FD020D497E00E5302532FFEE3541
:100BAC002FFEC3EF94E6EE940A5003020C6EEF9402
:100BBC0086EE94104003020C6EEF241AFBEE34F513
:100BCC00FA7C007D48AF03FE123589ED4C701CFC9D
:100BDC007D48AF03AE02123589AD077538087B032B
:100BEC007F6D1253DC8E5F8F60802F20412CAF32D3
:100BFC007E00E5302532CFEE352FCF241ACF34F5D9
:100C0C00FE7C007D48123589AD077538087B037F63
:100C1C006D1253DC8E5F8F60D241E4F5333044FDAE
:100C2C00125567AF327E00E5302532CFEE352FCF2F
:100C3C00241ACF34F5FE7C007D481235899002A031
:100C4C00EDF0E0FF5401FEC3EF9E25E02EF0E02511
:100C5C0060F582E4355FF583E493F5333044FD02AF
:100C6C000D497E00E5302532FFEE352FFEC3EF94A3
:100C7C0086EE94105003020D3AEF9426EE94164033
:100C8C0003020D3AEF247AFBEE34EFFA7C007D4838
:100C9C00AF03FE123589ED4C701CFC7D48AF03AEE2
:100CAC0002123589AD077538087B037F6D1253DC52
:100CBC008E5F8F60802F20412CAF327E00E5302577
:100CCC0032CFEE352FCF247ACF34EFFE7C007D4827
:100CDC00123589AD077538087B037F6D1253DC8E96
:100CEC005F8F60D241E4F5333044FD125567AF326B
:100CFC007E00E5302532CFEE352FCF247ACF34EF7E
:100D0C00FE7C007D481235899002A0EDF0E0FF5486
:100D1C0001FEC3EF9E25E02E2402F0E02560F58253
:100D2C00E4355FF583E493F5333044FD800FE4F54F
:100D3C00333044FD1255677533013044FD1255674D
:100D4C0005320203173044FD305F03020E11855A41
:100D5C0099C2443044FD855B99C244304403020E71
:100D6C001180F8900034E0FD64107043305F057F13
:100D7C000612534DE4F53274332532F582E4340017
:100D8C00F583E0F533F599C2443044FDAF33125589
:100D9C006E0532E532C3940640DD205F68855A99B2
:100DAC00C2443044FD855B99C24420445880FBED1D
:100DBC00641A7051305F057F0312534D900033E07D
:100DCC00F533853399C2443044FDAF3312556E90E0
:100DDC000034E0F533853399C2443044FDAF33120F
:100DEC00556E855E33853399C2443044FD205F15C2
:100DFC00AF3312556E855A99C2443044FD855B99C8
:050E0C00C2443044FD6A
:010E110022BE
:10198500753301C24A900034E0640660030220808A
:10199500A3E0FEA3E0FD7A002400FFEA3EFEC3EFCC
:1019A5009464EE648094804003021C04ED9401501D
:1019B500337B017A007938753901753A04753B0234
:1019C500753C00E4FF1251D17B017A0079377539F6
:1019D50001753A04753B02753C007F011251D143F4
:1019E5005D01805D900036E0D3940350337B017A2E
:1019F500007938753901753A04753B02753C007FED
:101A0500021251D17B017A007937753901753A0493
:101A1500753B02753C007F031251D1435D02802165
:101A2500900036E0640870307B017A0079387539AA
:101A350001753A04753B02F53C7F081251D1435DAF
:101A4500047B007A00795D753901753A04753B02AE
:101A5500753C007F63021BFE900036E0FF64047056
:101A6500030222B2EF640570030222B2EF6407702D
:101A7500030222B2EFB406157B017A007938753975
:101A850001753A04753B02753C00021BC490003693
:101A9500E0B40B177B017A007938753901753A0482
:101AA500753B02753C007F0B021BFE900036E0641F
:101AB5000C7032A3E0FEA3E07C002400F530EC3E80
:101AC500F52FC39400401BD3E5309401E52F940016
:101AD5005010E530452F9000297004F0021FB174B5
:101AE50001F0021FB1900036E0B40D227B017A00AF
:101AF5007938753901753A04753B02753C007F0DDF
:101B05001251D1900038E0900268F00222B29000A4
:101B150036E0640F703B7B017A00793875390175C1
:101B25003A04753B02F53C7F0F1251D1900038E025
:101B3500645560030222B2F532E532245BFF7D0174
:101B45001255031254AF0532E532D3941B40EA8097
:101B5500FE900036E064107042900038E0B4AA1B95
:101B65007D1C7F5B1255037520FF7521FF7522FFD4
:101B75007F887E13125694C2AF80FE7B017A00796E
:101B850038753901753A04753B02753C007F1012B2
:101B950051D1900038E0F5330222B2900036E0646E
:101BA5000A70339000D4E0640160030222B27B0125
:101BB5007A007938753901753A04753B02F53C7F31
:101BC500061251D1900038E0F55E7D067CEFE4FF0A
:101BD5001252CA0222B2900036E0FFB45A099000B0
:101BE50038E042260222B27B017A00793875390144
:101BF500753A04753B02753C001251D10222B29030
:101C05000035E0FEA3E0FD7A002400FFEA3EFEC3B6
:101C1500EF94C8EE6480948040030222B2EDC39431
:101C2500644008E0946A50030222B2900036E0FD59
:101C3500646A7047A3E0FEA3E07A002400F530EA69
:101C45003EF52F4530600BE5306401452F600302FA
:101C550022B2900038E090000FF064016003022288
:101C6500B275320774092532F582E43400F583E450
:101C7500F00532E532B413EC0222B2EDC3946B40A9
:101C85003E900036E0FD9477503590000FE0702FC0
:101C9500900037E0FEA3E07A002400F530EA3EF537
:101CA5002FD3E53094FFE52F940040030222B27450
:101CB500A52DF582E434FFF583E530F00222B290DC
:101CC5000036E0FD64777069A3E0FEA3E0FC7A00CE
:101CD5002400F530EA3EF52FC3940050030222B2EA
:101CE500D3E5309402E52F940040030222B2E09040
:101CF500001CF0701A75321674092532F582E43429
:101D050000F583E4F00532E532B41EEC0222B2ECB4
:101D1500640160030222B275321474092532F5821A
:101D2500E43400F583E4F00532E532B416EC022222
:101D3500B2ED6478703D90001CE064016035900060
:101D450037E0FDFEA3E0FC7A002400F530EA3EF51D
:101D55002FD3E5309400E52F940050030222B2D32F
:101D6500E53094FFE52F947F40030222B290001DD9
:101D7500021ED8900036E0FFC39479403DEF947D74
:101D8500503890001CE06032900037E0FEA3E0FD83
:101D95007A002400F530EA3EF52FD3E53094FFE5CF
:101DA5002F940040030222B2900036E024A6F5826B
:101DB500E434FFF583EDF00222B2900036E0F964D9
:101DC5007D703B90001CE06035900037E0FDFEA380
:101DD500E0FC7A002400F530EA3EF52FD3E5309497
:101DE50000E52F940050030222B2D3E53094FFE5BD
:101DF5002F947F40030222B2900023021ED8E9648B
:101E05007E703590001CE0602F900037E0FDFEA34A
:101E1500E0FC7A002400F530EA3EF52FC39400502B
:101E2500030222B2D3E53094FFE52F947F400302ED
:101E350022B2900025021ED8E9647F702E900037EB
:101E4500E0FDFEA3E0FC7A002400F530EA3EF52F24
:101E5500C3940050030222B2D3E53094FFE52F94DA
:101E65007F40030222B29000278068E96480702ACF
:101E7500900037E0FEA3E0FD7A002400F530EA3E4D
:101E8500F52FC394004010D3E5309401E52F94005D
:101E95005005900029EDF0021FB1900036E0F9647D
:101EA500817038A3E0FDFEA3E0FC7A002400F53044
:101EB500EA3EF52FC3E530940AE52F94005003025E
:101EC50022B2D3E5309488E52F941340030222B261
:101ED50090002AECF0A3EDF00222B2E96482706F63
:101EE500900037E0FEA3E07C002400F530EC3EF5E1
:101EF5002F4530704290002CE530F0C2A71254AF48
:101F0500E4900029F07B017A007929753901753A49
:101F150004753B02F53C7F0C1251D1C2CA75CDFF49
:101F250075CCB875CBFF75CAB8D2CA7F607EEA1288
:101F35005694D2A70222B2E5306401452F60030210
:101F450022B290002CE530F07889760202207A9052
:101F55000036E06483705CA3E0FEA3E07C0024000F
:101F6500F530EC3EF52FC3940050030222B2D3E5C1
:101F7500309403E52F940040030222B290002DE532
:101F850030F06401452F6008E5306403452F70117A
:101F9500E5306403452F7002D246E47889F60220C5
:101FA5007AE5306402452F60030222B27889760F04
:101FB50002207A900036E06484703BA3E0FEA3E043
:101FC5007C002400F530EC3EF52FC394005003024D
:101FD50022B2D3E5309401E52F940040030222B2EA
:101FE50090002EE530F06401452F60030222B2789F
:101FF50089760102207A900036E06485703AA3E084
:10200500FEA3E07C002400F530EC3EF52FC39400E0
:1020150050030222B2D3E5309401E52F940040032A
:102025000222B290002FE530F06401452F600302D3
:1020350022B278897603803D900036E064B960036A
:102045000222B2A3E0FEA3E07C002400F530EC3EC2
:10205500F52FC39400401AD3E5309401E52F940081
:10206500500FE530452F9000297003F0800374016F
:10207500F07889760F124D430222B2900034E06465
:102085001060030222B2A3E0FEA3E07C002400F569
:1020950030EC3EF52FE53064C8452F700C900038C4
:1020A500E0B408051247F9D257C3E530943CE52F53
:1020B50094035048C3E53094D0E52F9400403DE5A6
:1020C500302430FBE52F34FFFA7C007D1FAF03FE83
:1020D500123589ED4C60030222B2FC7D1FAF03AEC1
:1020E500021235898F32C2AC7B017A00793A753993
:1020F5001FE4F53A753B04F53C022206C3E530942E
:102105000CE52F94055049C3E530943CE52F940325
:10211500403EE53024C4FBE52F34FCFA7C007D1DF0
:10212500AF03FE123589ED4C60030222B2FC7D1D22
:10213500AF03AE021235898F32C2AC7B017A0079CA
:102145003A75391D753A01753B04753C0002220646
:10215500C3E5309406E52F94085055C3E530940C3B
:10216500E52F9405404AE53024F4FBE52F34FAFACF
:102175007C007D03AF03FE123589ED4C600302221E
:10218500B2FC7D03AF03AE021235898F32C2AC7B40
:10219500017A00793A753903753A02753B06753C43
:1021A500001251D1D2AC7D017F0412527F0222B2BE
:1021B500C3E53094E6E52F940A504EC3E530940606
:1021C500E52F94084043E53024FAFBE52F34F7FA70
:1021D5007C007D2EAF03FE123589ED4C6003022293
:1021E500B2FC7D2EAF03AE021235898F32C2AC7BB5
:1021F500017A00793A75392E753A03753B04753CB9
:10220500001251D1D2AC0222B2C3E5309486E52F3B
:102215009410504DC3E53094E6E52F940A4042E50D
:1022250030241AFBE52F34F5FA7C007D48AF03FE18
:10223500123589ED4C7076FC7D48AF03AE02123540
:10224500898F32C2AC753708753801753900753A12
:102255003A753B907B03AD327F6D123F2BD2AC803C
:102265004CC3E5309426E52F94165041C3E53094D0
:1022750086E52F94104036E530247AFBE52F34EFC0
:10228500FA7C007D48AF03FE123589ED4C701EFCCB
:102295007D48AF03AE021235898F32C2AC7B017A1D
:1022A50000793A7539907D031244ACD2ACE53364BC
:1022B5007F70367F777D01125503E4F5327D04AFDB
:1022C50032124AF08F828E83E493F531E42532FD94
:1022D500E434EEFCAF311252CA0532E532D3941024
:1022E50040DBC2AF759F8080FEE533B4FF07C2AF08
:0522F500759F8080FED2
:0122FA0022C1
:1048F6001256B61254AF9001D4E06401704D7B019C
:104906007A007933305F3DAD5012501A90029EEE18
:10491600F0A3EFF090029EE0FCA3E0FDECFF743301
:104926002550F582E43400F583EFF074342550F514
:1049360082E43400F583EDF0055005507B017A00E2
:1049460079338000AF5012537E804F9001D4E0FF40
:10495600B4021D125582E4FE74332EF582E434004F
:10496600F583E0F599C2443044FD0EBE08EA802A7C
:10497600EF6403702512388E501012558212028C85
:10498600C2411254AF1219858010305E04C21480E1
:1049960002C217E4FD7F0612527FC218E4FF1256C8
:0D49A6000FE4788AF69000D3F09001D4F071
:0149B30022E1
:104F41001255821254AF305F19156115619000D668
:104F5100E0B41909E561B40C0405610561AF6112A2
:104F6100534DE4FFEFC39561501574D52FF582E4DD
:104F71003400F583E0F599C2443044FD0F80E5D259
:0A4F8100AAD2A8C2197F0102560F40
:10564200900030E0B40108124F41E4900030F022A3
:0300230002297738
:10297700C0E0C0F0C083C082C0D075D000C000C026
:1029870001C002C003C004C005C006C007209803E9
:10299700022C1EC298E562B40231AF49054974D5CD
:1029A7002FF582E43400F583E599F0E549B4020593
:1029B7007F0512560F78877600087664205A03023F
:1029C7002C25187601087690022C25E562640160B3
:1029D70003022B51788AE6062433F582E43400F5A6
:1029E70083E599F0E6FF64017056305F3AF54AC215
:1029F70015C245755006900031F0A3740EF0900093
:102A0700D3E0FEC394064003022C25900033E0FD7B
:102A170074032EF582E43400F583EDF09000D3E0E3
:102A270004F07600022C25754B00C212C2479000B5
:102A3700D3E4F0900031F0A37408F0F550022C2590
:102A4700EF6402704B900033E0FFF46004EFB55E73
:102A570005755CA18003755CA2900034E0FF6419E2
:102A67006004EFB41A19305F057550048003755080
:102A770006D242EFB41905755CA28003755CA1907C
:102A87000034E064106003022C25755008022C25E1
:102A9700788AE6FC6407704B900034E0FDB41018A8
:102AA700900039E0FF2409F550EF2404FEE4339049
:102AB7000031F0A3CEF0801E900037E0B45517ED3B
:102AC700B40613900036E0B40A0C75500C90003130
:102AD700E4F0A37406F0205F03022C25155015506F
:102AE700022C25ECB55013900034E0FF64036025F9
:102AF700EF64066020EF6410601B788AE66550601B
:102B070003022C25900034E0FF64196008EF641A73
:102B17006003022C25E55CB4A1089001D47403F08E
:102B27008010E55C9001D4B4A2057401F0800374B1
:102B370004F0756200900031E4F0A3F0D218FDFFB5
:102B470012527FD247D245022C25E5626403600307
:102B5700022C25AF49054974D52FF582E43400F5D9
:102B670083E599F0E549B40111C20D75610890003C
:102B770001E4F0A37410F0022C25E5496403703DCD
:102B87009000D6E0FDB4031BA3E0FF2405F561EF39
:102B970075F004A42406FEE435F0900001F0A3CEFE
:102BA700F0807BED64196003304273C242D25275E4
:102BB700610C900001E4F0A3740CF08061E549B466
:102BC70006259000D9E0645570549000D6E064065D
:102BD700704C9000D8E0640A704475610C90000155
:102BE700F0A37407F08037E5496561703190000103
:102BF700F0A3F0F549C252D20D305608C256D2584A
:102C0700D259801AD2D8D219E4FD7F0112527F908F
:102C170000307401F08007309904C299D244D0077C
:102C2700D006D005D004D003D002D001D000D0D038
:092C3700D082D083D0F0D0E0324D
:0B56AB00C2A1D2A2D2A1C2A2C2A122C1
:0756BD00C2A2D2A1D2A22279
:0855AF001256AB7FA212562038
:0C55B700D2A2D2A1A2A2924BC2A1A24B90
:0155C30022C5
:105620007E08EF3392A2D2A1C2A1EF25E0FFDEF205
:015630002257
:1054DB00E4F53AF539D2A1E53A25E0FFA2A2E4338F
:1054EB004FF53AC2A17F017E001256940539E5397A
:0754FB00C3940840E0AF3A42
:015502002286
:0A4D9F008D348B358A368937AC0756
:104DA900C2AF1256BD1255AFAF041256201255B7F5
:104DB9001256AB7FA31256201255B7E4F538E538E1
:104DC900C3953450211254DBAB35AA36A93785383F
:104DD90082758300EF123555E53414653860031286
:0E4DE90055B7053880D81255B71256BDD2AF57
:014DF7002299
:10554A00AC07C2AF1255AFAF041256201255B7AF0F
:0D555A00051256201255B71256BDD2AF22D1
:1047F900900039E0FF900038E06F7073900041E05D
:10480900FF1255EAAD077F0212554A900040E0FFBA
:104819001255EAAD077F0312554A90003FE0FF1297
:1048290055EAAD077F0412554A90003EE0FF125544
:10483900EAAD077F0512554A90003DE0FF1255EA9F
:10484900AD077F0612554A90003AE090003CB41338
:1048590006E04480F08004E0547FF090003CE0FFE3
:104869001255EAAD077F0712554A90003B807190B7
:104879000049E0FF1255EAAD077F0212554A900040
:1048890047E0FF1255EAAD077F0312554A900045EC
:10489900E0FF1255EAAD077F0412554A900043E044
:1048A900FF1255EAAD077F0512554A900041E0FF16
:1048B9001255EAAD077F0612554A90003BE0900079
:1048C9003FB41306E04480F08004E0547FF0900088
:1048D9003FE0FF1255EAAD077F0712554A90003DA8
:0D48E900E0FF1255EAAD077F0812554A2284
:10522D0001820A012500012700012400012600C189
:01523D005719
:10563100EFC4540FFEEF540FFFEE75F00AA42FFFD5
:015641002246
:1055EA00EF75F00A84FEEF75F00A84EEC454F025D4
:0255FA00F0FFC0
:0155FC00228C
:102660007B007A0079327D017F08124D9FAF3212D4
:1026700056318F327B007A0079317D017F07124D10
:102680009FE53130E706E532246C8004E53224D042
:10269000F530E43407F52F53311F7B007A0079328F
:1026A0007D017F05124D9F53323FAF321256318F5D
:1026B000327B007A0079847D017F06124D9F7884F9
:1026C000E65407F67B007A0079837D017F04124D82
:1026D0009F7883E6543FF6E6FF125631A6077B004B
:1026E0007A0079817D017F03124D9F7881E6547FC6
:1026F000F6E6FF125631A60790027CE06401700BEB
:102700007883E6C39402403B06801190027CE0642B
:102710000270307883E6C39402402816E6FF125513
:10272000EAAD077F0412554AE490027CF07B017AFF
:1027300002797C753901753A04753B02F53C7F0ED0
:102740001251D17884E6FF78826670062057030222
:1027500029767882A607C257E53112368D27850182
:1027600027910227980327E704283F0528510628C8
:10277000630728750828870928A11028FF11295602
:10278000120000296EAF327885760008A60702296C
:102790006EE532241F022897E53054037006E532B7
:1027A000243C8004E532243B7886F6E43318F69026
:1027B0000268E06401600302296EC3E53094D7E546
:1027C0002F9407500302296EE53294085003022922
:1027D0006EE532D3940E400302296E7884E66406D7
:1027E000600302296E8043E53054037006E532240D
:1027F0005B8004E532245A7886F6E43318F69002BA
:1028000068E06401600302296EC3E53094D7E52FC8
:102810009407400302296EE5329407400302296EB3
:102820007884E66406600302296E90027C04F0FB63
:102830007A02797CF539753A04753B0202294CE538
:102840003054037006E53224798004E53224788020
:1028500046E53054037006E53224988004E53224BE
:10286000978034E53054037006E53224B68004E5E1
:102870003224B58022E53054037006E53224D58039
:1028800004E53224D48010E53054037006E5322488
:10289000F48004E53224F37886F6E43318F602294E
:1028A0006EE53054037006E53224128004E53224CC
:1028B000117886F6E4340118F6900268E06401604D
:1028C0000302296EC3E53094D7E52F940740030235
:1028D000296EC3741F9532D39406400302296E7883
:1028E00084E66406600302296E90027C7402F07B29
:1028F000017A02797C753901753A04F53B804DE522
:102900003054037006E53224318004E532243078F7
:1029100086F6E4340118F6900268E06401704FC353
:10292000E53094D7E52F94074044E532D39407501F
:102930003D7884E66406703690027C7402F07B0178
:102940007A02797C753901753A04F53B753C007F54
:102950000E1251D18018E53054037006E532244F31
:102960008004E532244E7886F6E4340118F6788641
:06297000E61618700116C6
:01297600223E
:10543400E52F5407FFE52F131313541F7C00244852
:07544400F9EC3402FA7B01D0
:10544B007E01EEA807088002C333D8FCFE1234FDA0
:04545B004E02354385
:10540800E5325407FFE532131313541F7C00241BA5
:05541800F9EC3402FA7A
:10541D007E01EEA807088002C333D8FCFE6306FFA9
:07542D001234FD5E0235435D
:0853AE007A0279457B01AF3062
:1053B6007E01EF131313541FFDEF5407FFEEA807EA
:1053C600088002C333D8FCFEAF058F8275830012B6
:0553D60035165E24FF06
:0153DB0022AF
:1045E900E4F52F7D01AF2F124AF08F828E83741C60
:1045F90093F527303F0302468F7530017885E6FC35
:1046090008E6FDAE047803CEC313CE13D8F9F5310D
:10461900ED5407FFE530A807088002C333D8FCF53D
:10462900307D03AF2F124AF08F828E83740B93F47F
:104639006038742693F46032E5822531F582E435D9
:1046490083F583E493553060127B017A02793BAF9D
:104659002F1253B650030246E780407B017A027954
:104669003BAF2F1253B65076805AE52F5407FFE51A
:104679002F131313541F7C00243BF9EC3402FA7BEB
:104689000112541D8058E527F46053303E297B01FF
:104699007A02793BAF2F1253B64043E52F5407FFF7
:1046A900E52F131313541F7C00243BF9EC3402FA51
:1046B90012544BC23180277B017A02793BAF2F120A
:1046C90053B6501AE52F5407FFE52F131313541F40
:1046D9007C00243BF9EC3402FA12541DC231052F37
:0A46E900E52FC3941050030245ECC6
:0146F30022A4
:102C4000E4F5307884E6F52FC394005003752F0621
:102C5000E4FDAF30124AF08E328F338F828E837450
:102C60001E93F525741D93F531D364809480500331
:102C7000022D04D3E531648094904003022D0415A5
:102C800031753401E5315407FFE534A807088002A7
:102C9000C333D8FCF534E5317803A2E713D8FBFF42
:102CA0003395E0FE743B2FF58274023EF583E055C8
:102CB0003460287A0279181253B2401AE53054076A
:102CC000FFE530131313541F7C002418F9EC340271
:102CD000FA12544BC230752F0880437B017A027977
:102CE00018AF301253B65036E5305407FFE53013B5
:102CF0001313541F7C002418F9EC3402FA12541DEB
:102D0000C230801AE5305407FFE530131313541F07
:102D10007C002418F9EC3402FA7B0112541D85332F
:102D200082853283741C93F531D364809480500380
:102D3000022DC8D3E531648094904003022DC8155C
:102D400031753401E5315407FFE534A807088002E6
:102D5000C333D8FCF534E5317803A2E713D8FBFF81
:102D60003395E0FE743B2FF58274023EF583E05507
:102D700034602C7B017A027915AF301253B6401AB9
:102D8000E5305407FFE530131313541F7C0024155E
:102D9000F9EC3402FA12544BC230752F0780437B92
:102DA000017A027915AF301253B65036E530540728
:102DB000FFE530131313541F7C002415F9EC340283
:102DC000FA12541DC230801AE5305407FFE5301363
:102DD0001313541F7C002415F9EC3402FA7B011202
:102DE000541D302F03022E6E7538087B03AD307FE3
:102DF0006D1253DC8E328F33E52F75F010A425331E
:102E0000FFE5F03532CF240ECF3400FE7531078F49
:102E1000828E83E493FD70040493601C7883E6FC47
:102E2000D39D50278F828E83E493B5040B74019356
:102E3000FD7881E6C39D501374FE2FFF74FF3EFEA4
:102E40001531C3E5316480948050C4C3E53164809A
:102E5000948050071253AE505D8041E53130E00759
:102E60001253AE505180351253AE404A800DE525C5
:102E7000F46043302E211253AE403BE5305407FF3F
:102E8000E530131313541F7C002445F9EC3402FA87
:102E900012544BC230801F1253AE501AE530540703
:102EA000FFE530131313541F7C002445F9EC340262
:102EB000FA12541DC2300530E530C3941450030299
:022EC0002C43A1
:012EC20022ED
:04436A009250AF2F8F
:02436E008F328C
:10437000753503C2510532AF351535EF7003024470
:10438000643050089000D97401F08005E49000D9A1
:10439000F090023DE532F0A37406F09000D9E09071
:1043A0000242F07B017A02793D7D0612501A8E336B
:1043B0008F34900243E533F0A3E534F07B017A02B9
:1043C000793D7F0812537ED256C258C259C28EE43C
:1043D000F58DF58BD28EF533205920E58DD394D809
:1043E00040F61254AFC28EE4F58DF58BD28E0533B4
:1043F000E533C3940640E1D259C2589000D5E06538
:104400003260030243772058030243777B017A002E
:1044100079D57D08124EF5400302437715323050AE
:10442000297B017A02791BAF321253B6402EE53256
:104430005407FFE532131313541F7C00241BF9ECBF
:104440003402FA12544BC23280127B017A02791B79
:10445000AF321253B65005125408C232E4F535D2C9
:1044600051024377E535F4704220513F1532305008
:10447000287B017A02791BAF321253B6402DE53208
:104480005407FFE532131313541F7C00241BF9EC6F
:104490003402FA12544BC232227B017A02791BAFEA
:0B44A000321253B65005125408C2320D
:0144AB0022EE
:10330B00C24AC24BC24CE4F52F1254AFC2AC7D0281
:10331B00AF2F124AF08E308F31D2ACEF64DC7003DA
:10332B00EE64B470030234F08F828E83740293F5D3
:10333B0024C24EC24FE493FFD39400406AEFD39460
:10334B00145064EF14FF7B017A0279451253B65087
:10335B0029D24A7A0179D5AF2F1253B64045E52FC2
:10336B005407FFE52F131313541F7C0024D5F9ECDE
:10337B003401FA12544BC2328029C24A7B017A01C2
:10338B0079D5AF2F1253B6501AE52F5407FFE52FFF
:10339B00131313541F7C0024D5F9EC3401FA125487
:1033AB001DC232D24E801AE52F5407FFE52F13139F
:1033BB0013541F7C0024D5F9EC3401FA7B01125411
:1033CB001D853182853083740193FFD39400406A4D
:1033DB00EFD394145064EF14FF7B017A02794512FA
:1033EB0053B65029D24B7A0179F5AF2F1253B64011
:1033FB0045E52F5407FFE52F131313541F7C0024AF
:10340B00F5F9EC3401FA12544BC2328029C24B7BD2
:10341B00017A0179F5AF2F1253B6501AE52F5407E5
:10342B00FFE52F131313541F7C0024F5F9EC340123
:10343B00FA12541DC232D24F801AE52F5407FFE502
:10344B002F131313541F7C0024F5F9EC3401FA7B72
:10345B000112541D20274E204E06204F030234F03C
:10346B007B017A02791BAF2F1253B6924C7A0279F9
:10347B0048AF2F1253B6924DA24B724A304C01B348
:10348B004003204D0C204D03125434A24B724A8042
:10349B0040305551A24B724A12436AE52F64FD70BE
:1034AB0044C2558040E524F4603B7B017A027948A5
:1034BB00AF2F1253B6924D7A02791BAF2F1253B620
:1034CB00302601B34003204D0D204D03125434A27E
:1034DB002612436A800F30550CA22612436AE52F41
:1034EB00B4FD02C255052FE52FC394FE50030233E2
:0134FB0014BC
:0134FC0022AD
:1049B40061646D696E00736574206970200073749E
:1049C40061746963200073657420686F73742000D8
:1049D4007463707320007463706320007463707375
:1049E4006320007365742073657269616C203936C5
:1049F4003030202A202A202A202A202A202A200077
:104A04007365742073657269616C2031393230309A
:104A1400202A202A202A202A202A202A20006765EA
:104A24007420737461747573006765742069700011
:104A340067657420686F73740067657420736572AA
:104A440069616C00736176650065786974007265EC
:104A5400626F6F7400666163746F72796465666116
:044A6400756C7400F9
:09523E00C15BC1DAC15D0115007C
:0F565200C2A8C2AAD21AC295C297D2A3D2A422CA
:0F566100E4F549D2D8D2D9756202C295C2972218
:104F8B00C2D8C2D9D295E4900000F0F5627D047FBF
:104F9B000C124AF08F828E83E493B40112C2CA754D
:104FAB00CDFF75CCDC75CBFF75CADCD2CA8010C2C5
:104FBB00CA75CDFF75CCB875CBFF75CAB8D2CAC24E
:0A4FCB001AD2A8D2AA7F0502560FE1
:1050A0001256617512FF7513497514B4AB12AA1329
:1050B000A9141234FD60160514E5147002051314CA
:1050C000F91234FDF599C2442044E180FB75990D35
:0D50D000C244E4FD7F0512527F3044FD22F2
:104D4300E4F515C25A900000F0FF12560F125652A6
:104D5300125661C2CA75CDFF75CCB875CBFF75CA43
:104D6300B8D2CAD2927F507EC31256941254AF7FE8
:104D7300507EC3125694C2921254AF7F507EC31218
:104D830056941254AF7F507EC312569475990DC238
:0C4D930044E4FD7F0512527F3044FD22F5
:1042160090001EE090001DFEE07C002400FFEC3EB6
:01422600FE99
:044227008E328F3311
:10422B00D3E5339409E5329400500D753401EF2436
:10423B0030900033F0024353D3E5339463E532946B
:10424B00005038E4F534AE32AF337C007D0A1235C2
:10425B0089ED2430FF74332534F582E43400F58383
:10426B00EFF0AE32AF337C007D0A1235898E328F80
:10427B00330534E534B402CE024353D3E53394E72C
:10428B00E53294035038E4F534AE32AF337C007D25
:10429B000A123589ED2430FF74332534F582E4346A
:1042AB0000F583EFF0AE32AF337C007D0A12358917
:1042BB008E328F330534E534B403CE024353D3E54A
:1042CB0033940FE53294275037E4F534AE32AF33E5
:1042DB007C007D0A123589ED2430FF74332534F5CB
:1042EB0082E43400F583EFF0AE32AF337C007D0A0D
:1042FB001235898E328F330534E534B404CE8048C1
:10430B00AE32AF33E4FCFD7BFF7AFFF9F8C3123614
:10431B00774035E4F534AE32AF337C007D0A12358D
:10432B0089ED2430FF74332534F582E43400F583B2
:10433B00EFF0AE32AF337C007D0A1235898E328FAF
:10434B00330534E534B405CE74322534F582E434C8
:0E435B0000F583E0F599C2443044FDD534EA04
:014369002231
:10545F007512FF7513497514BAAB12AA13A914125A
:10546F0034FD60160514E5147002051314F9123497
:0B547F00FDF599C2442044E180FB22AF
:104C75008F3174092FF582E43400F583E0FF7E005F
:104C850012422775992EC2443044FD740A2531F528
:104C950082E43400F583E0FF7E0012422775992EE9
:104CA500C2443044FD740B2531F582E43400F583AC
:104CB500E0FF7E0012422775992EC2443044FD74F0
:104CC5000C2531F582E43400F583E0FF7E001242C5
:0A4CD50027759920C2443044FD22E7
:104BF70012566112545F90000FE0703B7512FF75FB
:104C070013497514C2AB12AA13A9141234FD601606
:104C17000514E5147002051314F91234FDF599C251
:104C2700442044E180FB7F07124C757F0B124C75C3
:104C37007F0F124C75802890000FE064017020757B
:104C47009964C2443044FD759968C2443044FD7587
:104C57009963C2443044FD759970C2443044FD7570
:0E4C6700990DC2443044FDE4FD7F0502527FEA
:1040B9001256617512FF7513497514CAAB12AA130A
:1040C900A9141234FD60160514E5147002051314C1
:1040D900F91234FDF599C2442044E180FB90001C9B
:1040E900E070477512FF7513497514D4AB12AA1302
:1040F900A9141234FD60160514E514700205131491
:10410900F91234FDF599C2442044E180FB124216AC
:10411900759920C2443044FD900028E09000271290
:10412900421D759920C2443044FD90001CE0640191
:1041390070587512FF7513497514DAAB12AA13A9D1
:10414900141234FD60160514E5147002051314F9F0
:104159001234FDF599C2442044E180FB7F16124CCC
:1041690075900024E0FE90002312421E759920C22A
:10417900443044FD900026E0FE90002512421E7551
:104189009920C2443044FD0241FB90001CE06402C6
:10419900706B7512FF7513497514E0AB12AA13A958
:1041A900141234FD60160514E5147002051314F990
:1041B9001234FDF599C2442044E180FB1242167580
:1041C9009920C2443044FD7F16124C75900024E0BA
:1041D900FE90002312421E759920C2443044FD907E
:1041E9000026E0FE90002512421E759920C2443037
:1041F90044FD900028E0FE90002712421E75990D9B
:0D420900C244E4FD7F0512527F3044FD22C7
:104DF800125661900029E0700B7512FF7513497502
:104E080014E780097512FF75134A751404AB12AACA
:104E180013A9141234FD60160514E5147002051365
:104E280014F91234FDF599C2442044E180FB900046
:104E38002BE0FE90002A12421E75990DC244E4FD33
:094E48007F0512527F3044FD2267
:1050DD001256617512FF75134A751422AB12AA137D
:1050ED00A9141234FD60160514E51470020513148D
:1050FD00F91234FDF599C2442044E180FB75990DF8
:0D510D00C244E4FD7F0512527F3044FD22B4
:10511A001256617512FF75134A75142DAB12AA1334
:10512A00A9141234FD60160514E51470020513144F
:10513A00F91234FDF599C2442044E180FB75990DBA
:0D514A00C244E4FD7F0512527F3044FD2277
:105157001256617512FF75134A751434AB12AA13F0
:10516700A9141234FD60160514E514700205131412
:10517700F91234FDF599C2442044E180FB75990D7D
:0D518700C244E4FD7F0512527F3044FD223A
:105194001256617512FF75134A75143DAB12AA13AA
:1051A400A9141234FD60160514E5147002051314D5
:1051B400F91234FDF599C2442044E180FB75990D40
:0D51C400C244E4FD7F0512527F3044FD22FD
:064FD5009000007406F0DC
:104FDB00125661D25A7512FF75134A751448AB12EB
:104FEB00AA13A9141234FD60160514E514700205FA
:104FFB001314F91234FDF599C2442044E180FB757A
:0F500B00990DC244E4FD7F0512527F3044FD220F
:10505D001256617512FF75134A75144DAB12AA13D2
:10506D00A9141234FD60160514E51470020513140D
:10507D00F91234FDF599C2442044E180FB75990D78
:10508D00C244E4FD7F0512527F3044FD9000007450
:03509D000DF022F1
:1052E9007512FF75134A751452AB12AA13A9141239
:1052F90034FD60160514E5147002051314F912340F
:10530900FDF599C2442044E180FB75990DC24430F2
:0353190044FD222E
:104CDF001256617512FF75134A751459AB12AA1348
:104CEF00A9141234FD60160514E51470020513148F
:104CFF00F91234FDF599C2442044E180FB90002C59
:104D0F00E064017020759920C2443044FD75992DDF
:104D1F00C2443044FD759969C2443044FD759970A1
:104D2F00C2443044FD75990DC2443044FDE4FD7F0B
:044D3F000502527F98
:093A3D00900027EFF0AD2FAF302F
:023A4600A907CE
:103A4800ED24FE7003023BC8147003023B9414700B
:103A580003023B50147003023AEB146003023BDE8E
:103A680074D629F582E43400F583E024D0FFE434E9
:103A7800FFFE7C037DE8123577AA06AB0774D529CB
:103A8800F582E43400F583E024D0FFE434FFFE7CC3
:103A9800277D10123577EF2BFBEE3AFA74D729F50C
:103AA80082E43400F583E024D0FFE434FFFE7C0098
:103AB8007D64123577EF2BFBEE3AFA74D829F5823C
:103AC800E43400F583E024D0FFE434FFFE7D0A12DD
:103AD8003577EF2BFFEE3AFE74D929F582E43400EE
:103AE800023BB574D629F582E43400F583E024D08E
:103AF800FFE434FFFE7C007D64123577AA06AB072D
:103B080074D529F582E43400F583E024D0FFE43449
:103B1800FFFE7C037DE8123577EF2BFBEE3AFA7453
:103B2800D729F582E43400F583E024D0FFE434FF9C
:103B3800FE7C007D0A123577EF2BFFEE3AFE74D833
:103B480029F582E43400806574D629F582E43400CE
:103B5800F583E024D0FFE434FFFE7C007D0A1235B3
:103B680077AA06AB0774D529F582E43400F583E01B
:103B780024D0FFE434FFFE7D64123577EF2BFFEE8F
:103B88003AFE74D729F582E43400802174D529F5EA
:103B980082E43400F583E024D0FFE434FFFE7C00A7
:103BA8007D0A12357774D629F582E43400F583E06E
:103BB80024D0FDEC34FFCD2FF532ED3EF531801BDE
:103BC80074D529F582E43400F583E024D0F532E495
:0F3BD80034FFF5318005E4F531F532AE31AF320F
:013BE70022BB
:100E1200C25C900000E014B40E00400302197B9003
:100E22000E2F75F003A4C58325F0C58373020E59F6
:100E3200020E7F020EA9020F86020FC402100302E5
:100E4200103C0210FD0212EE0214FD0218370219C4
:100E52002702197B0218F6E549B4091E9000D7E073
:100E6200B46C17A3E0B46F12A3E0B4670D90000056
:100E72007401F01250A0751509220212EBE549B473
:100E8200111E9000DCE0B47017A3E0B46112A3E07D
:100E9200B4730D9000007402F01250A075150B226D
:100EA20012505D75150C22E549642C6003020F8017
:100EB2009000E2E064686003020F80A3E064656072
:100EC20003020F80A3E0646C6003020F807889E65E
:100ED20070099000007403F0024BF77889E6B40FB2
:100EE200099000007405F0024DF87889E6B40124F7
:100EF200752F077409252FF582E43400F583E4F099
:100F0200052FE52FB427EC9000007407F01250DD96
:100F120075150D227889E6B4020D900000740BF06D
:100F2200124CDF75150F227889E6640360030219FB
:100F3200841252E97F507EC31256941254AF7F50EE
:100F42007EC31256941254AF7F507EC3125694122F
:100F520054AF7F507EC31256941254AF7F507EC35B
:100F62001256941254AF7F507EC31256941254AF4D
:100F72007F507EC3125694124F8B75151022751531
:100F820011021978E549D39405400674FB2549F509
:100F92004974D52549F582E43400F583E0B44B1C4D
:100FA20074D42549F582E43400F583E0B44F0D9002
:100FB20000007404F01240B9751501227515020281
:100FC2001978E549D39405400674FB2549F549741F
:100FD200D52549F582E43400F583E0B44B1C74D482
:100FE2002549F582E43400F583E0B44F0D9000000A
:100FF2007405F0124DF87515032212505D75150433
:1010020022E549D39405400674FB2549F54974D578
:101012002549F582E43400F583E0B44B1674D425F7
:1010220049F582E43400F583E0B44F07124FD575D9
:1010320015052212505D75150622E549D394054027
:101042000674FB2549F54974D52549F582E4340037
:10105200F583E0644B60030210F674D42549F582EF
:10106200E43400F583E0644F60030210F67B017AFA
:10107200007929753901753A04753B02F53C7F0CFC
:101082001251D11252E9900029E07012C2CA75CDF4
:10109200FF75CCB875CBFF75CAB8D2CA8010C2CA68
:1010A20075CDFF75CCDC75CBFF75CADCD2CA7F501B
:1010B2007EC31256941254AF7F507EC312569412BE
:1010C20054AF7F507EC31256941254AF7F507EC3EA
:1010D2001256941254AF7F507EC31256941254AFDC
:1010E200124F8BE47887F608F6304604C246D25D8A
:1010F2007515072212505D751508229000FFE064F5
:101102004D60030212EBA3E0644160030212EBA301
:10111200E0644360030212EB90010CE0D394394087
:1011220005E024A9800690010CE024D0C454F0FF0D
:1011320090010DE0D394394006E024A9FE80079087
:10114200010DE024D0FEEF2E900009F090010FE097
:10115200D394394005E024A9800690010FE024D001
:10116200C454F0FF900110E0D394394006E024A962
:10117200FE8007900110E024D0FEEF2E90000AF0CE
:10118200900112E0D394394005E024A98006900131
:1011920012E024D0C454F0FF900113E0D3943940FC
:1011A20006E024A9FE8007900113E024D0FEEF2E72
:1011B20090000BF0900115E0D394394005E024A98A
:1011C2008006900115E024D0C454F0FF900116E08F
:1011D200D394394006E024A9FE8007900116E0244A
:1011E200D0FEEF2E90000CF0900118E0D39439401D
:1011F20005E024A98006900118E024D0C454F0FF31
:10120200900119E0D394394006E024A9FE800790AA
:101212000119E024D0FEEF2E90000DF090011BE0AA
:10122200D394394005E024A9800690011BE024D024
:10123200C454F0FF90011CE0D394394006E024A985
:10124200FE800790011CE024D0FEEF2E90000EF0ED
:10125200E4F52FAF2F052F743D2FF582E43401F50D
:1012620083E0B42EEEE52F2468F530AD2F7F6812AF
:101272003A46900010EFF0E4F52FAF2F052FE5303E
:101282002F24D5F582E43400F583E0B42EEC123A33
:1012920042900011EFF0E52F2530F530E4F52FAF45
:1012A2002F052FE5302F24D5F582E43400F583E0B5
:1012B200B42EEC123A42900012EFF0E52F2530F5F1
:1012C20030E4F52FAF2F052FE5302F24D5F582E43A
:1012D2003400F583E0B40DEC123A42900013EFF0C3
:1012E2009000007408F002511A0219789000E6E0AA
:1012F200647360030214DAA3E0647460030214DA14
:10130200A3E0646160030214DA90000FF0F52FAFDE
:101312002F052F74FA2FF582E43400F583E0B42E02
:10132200EEE52F2425F530AD2F7F25123A469000A9
:1013320010EFF0E4F52FAF2F052FE5302F24D5F570
:1013420082E43400F583E0B42EEC123A42900011AC
:10135200EFF0E52F2530F530E4F52FAF2F052FE51F
:10136200302F24D5F582E43400F583E0B42EEC125C
:101372003A42900012EFF0E52F2530F530E4F52FD8
:10138200AF2F052FE5302F24D5F582E43400F58305
:10139200E0B40DEC123A42900013EFF0E52F253045
:1013A200F530E4F52F740E2530F530AF2F052FE51B
:1013B200302F24D5F582E43400F583E0B42EEC120C
:1013C2003A42900014EFF0E52F2530F530E4F52F86
:1013D200AF2F052FE5302F24D5F582E43400F583B5
:1013E200E0B42EEC123A42900015EFF0E52F2530D2
:1013F200F530E4F52FAF2F052FE5302F24D5F582F8
:10140200E43400F583E0B42EEC123A42900016EF79
:10141200F0E52F2530F530E4F52FAF2F052FE5301D
:101422002F24D5F582E43400F583E0B40DEC123AB2
:1014320042900017EFF0E52F2530F530E4F52F74D8
:101442000A2530F530AF2F052FE5302F24D5F58250
:10145200E43400F583E0B42EEC123A42900018EF27
:10146200F0E52F2530F530E4F52FAF2F052FE530CD
:101472002F24D5F582E43400F583E0B42EEC123A41
:1014820042900019EFF0E52F2530F530E4F52FAF4B
:101492002F052FE5302F24D5F582E43400F583E0C3
:1014A200B42EEC123A4290001AEFF0E52F2530F5F7
:1014B20030E4F52FAF2F052FE5302F24D5F582E448
:1014C2003400F583E0B40DEC123A4290001BEFF0C9
:1014D200E52F2530F53080179000E6E0B46419A3BB
:1014E200E0B46814A3E0B4630F90000F7401F090AD
:1014F20000007409F00251570219789000EDE0647F
:1015020073706DA3E0640D706790001CF0F52FAF4F
:101512002F052F74FC2FF582E43400F583E0B40D1F
:10152200EEE52F2427F530AD2F7F27123A46EF90B4
:10153200001DF0AD2F7F27123A46EE90001EF0E418
:10154200F52F741A2530F530AF2F052FE5302F24F3
:10155200D5F582E43400F583E0B40DEC123A421280
:101562003A3DEE900028F0E52F2530F53002182B99
:101572009000EDE0646360030216AFA3E0640D60C7
:10158200030216AF90001C04F0E4F52FAF2F052FD5
:1015920074002FF582E43401F583E0B42EEEE52FDA
:1015A200242BF530AD2F7F2B123A4690001FEFF01F
:1015B200E4F52FAF2F052FE5302F24D5F582E43443
:1015C20000F583E0B42EEC123A42900020EFF0E5F1
:1015D2002F2530F530E4F52FAF2F052FE5302F24DE
:1015E200D5F582E43400F583E0B42EEC123A429051
:1015F2000021EFF0E52F2530F530E4F52FAF2F0570
:101602002FE5302F24D5F582E43400F583E0B40DC4
:10161200EC123A42900022EFF0E52F2530F530E44B
:10162200F52F74132530F530AF2F052FE5302F2419
:10163200D5F582E43400F583E0B40DEC123A429021
:101642000023123A40EE900024F0E52F2530F530C9
:10165200E4F52F74222530F530AF2F052FE5302F1A
:1016620024D5F582E43400F583E0B40DEC123A425D
:10167200EF900025123A41EE900026F0E52F25303A
:10168200F530E4F52F741A2530F530AF2F052FE52C
:10169200302F24D5F582E43400F583E0B40DEC124A
:1016A2003A42123A3DEE900028F002182B9000EDDB
:1016B200E064736003021834A3E0646360030218F9
:1016C20034A3E0640D600302183490001C7402F02D
:1016D200E4F52FAF2F052F74FD2FF582E43400F5CA
:1016E20083E0B40DEEAD2F7F28123A46EF90001D35
:1016F200F0AD2F7F28123A46EE90001EF0E52F241F
:1017020028F530E4F52F74112530F530AF2F052F71
:10171200E5302F24D5F582E43400F583E0B42EECD5
:10172200123A4290001FEFF0E52F2530F530E4F534
:101732002FAF2F052FE5302F24D5F582E43400F5A5
:1017420083E0B42EEC123A42900020EFF0E52F2510
:1017520030F530E4F52FAF2F052FE5302F24D5F5E6
:1017620082E43400F583E0B42EEC123A4290002178
:10177200EFF0E52F2530F530E4F52FAF2F052FE5FB
:10178200302F24D5F582E43400F583E0B40DEC1259
:101792003A42900022EFF0E52F2530F530E4F52FA4
:1017A20074132530F530AF2F052FE5302F24D5F5F2
:1017B20082E43400F583E0B40DEC123A42EF90007B
:1017C20023123A41EE900024F0E52F2530F530E463
:1017D200F52F74222530F530AF2F052FE5302F2459
:1017E200D5F582E43400F583E0B40DEC123A42EF11
:1017F200900025123A41EE900026F0E52F2530F5B3
:1018020030E4F52F741A2530F530AF2F052FE5306F
:101812002F24D5F582E43400F583E0B40DEC123ABE
:1018220042123A3DEE900028F0900000740AF00255
:1018320051940219789000E1E0644260030218EFCB
:10184200A3E0646160030218EFA3E0647560030221
:1018520018EFF52FAF2F052F74EB2FF582E434002C
:10186200F583E0B40DEEAD2F7F16123A46BE251E6B
:10187200BF801B900029E06035E4F07B017A00799B
:1018820029753901753A04753B02F53C801B9000BD
:1018920029E0640160187401F0FB7A007929F539B6
:1018A200753A04753B02753C007F0C1251D1E52F4D
:1018B2002416F530E4F52F748A2530F530AF2F0564
:1018C2002FE5302F24D5F582E43400F583E0B40D02
:1018D200EC123A42EF90002A123A41EE90002BF0BD
:1018E200900000740DF012505D7515122212505DB9
:1018F20075151322E549D394054002154974D5257F
:1019020049F582E43400F583E0B44B1774D42549D9
:10191200F582E43400F583E0B44F0874642515F5CC
:1019220015D25B8054E549D39405400674FB2549E2
:10193200F54974D52549F582E43400F583E0644B1A
:10194200703174D42549F582E43400F583E0B44F54
:1019520022E4900029F07B017A007929753901751A
:101962003A04753B02F53C7F0C1251D1124FD575EA
:1019720015142275151502505D124F8BE47887F607
:0219820008F665
:011984002240
:03000000020200F9
:0C020000787FE4F6D8FD75818B02024780
:1034FD00BB010689828A83E0225002E722BBFE02CD
:09350D00E32289828A83E49322FF
:10351600BB010CE58229F582E5833AF583E022506A
:1035260006E92582F8E622BBFE06E92582F8E222B4
:0D353600E58229F582E5833AF583E49322CE
:10354300BB010689828A83F0225002F722BBFE0167
:02355300F32261
:10355500F8BB010DE58229F582E5833AF583E8F0AC
:10356500225006E92582C8F622BBFE05E92582C858
:02357500F22240
:10357700EF8DF0A4A8F0CF8CF0A428CE8DF0A42E68
:02358700FE2222
:10358900BC000BBE0029EF8DF084FFADF022E4CC26
:10359900F875F008EF2FFFEE33FEEC33FCEE9DECEF
:1035A900984005FCEE9DFE0FD5F0E9E4CEFD22ED35
:1035B900F8F5F0EE8420D21CFEADF075F008EF2F7F
:1035C900FFED33FD4007985006D5F0F222C398FD70
:0535D9000FD5F0EA220D
:1035DE00C2D5EC30E709B2D5E4C39DFDE49CFCEE08
:1035EE0030E715B2D5E4C39FFFE49EFE123589C3C2
:1035FE00E49DFDE49CFC800312358930D507C3E4BD
:06360E009FFFE49EFE2276
:10361400BB010A89828A83E0F5F0A3E02250068781
:10362400F009E71922BBFE07E3F5F009E319228943
:0B363400828A83E493F5F07401932276
:10363F00BB010789828A830236B3500B09C5F02775
:10364F00F7C5F01937F722BBFE0D09F8E325F0F3A4
:10365F00C5F019E338F322F889828A837401932520
:08366F00F0C5F0F8E4933822E5
:10367700EB9FF5F0EA9E42F0E99D42F0EC6480C8CA
:0636870064809845F0226A
:10368D00D083D082F8E4937012740193700DA3A3CC
:10369D0093F8740193F5828883E4737402936860E0
:0636AD00EFA3A3A380DFE0
:104EA800AC16AD17AE18AF197810EC4D4E4F700414
:104EB8007CA57DA5C3EC13FCED13FDEE13FEEF13EB
:104EC800FF5010EC64CCFCED644CFDEE644EFEEF3C
:104ED80064CEFFD8DF8C168D178E188F19EE547F8D
:0D4EE800FE228E168F1774A5F518F51922FD
:10020C000236C9E493A3F8E493A34003F68001F209
:10021C0008DFF48029E493A3F85407240CC8C333F3
:10022C00C4540F4420C8834004F456800146F6DFC2
:10023C00E4800B010204081020408090520DE47EF3
:10024C00019360BCA3FF543F30E509541FFEE493B7
:10025C00A360010ECF54C025E060A840B8E493A37E
:10026C00FAE493A3F8E493A3C8C582C8CAC583CAA9
:10027C00F0A3C8C582C8CAC583CADFE9DEE780BE61
:015247000066
:1036B300C5F0F8A3E028F0C5F0F8E58215827002A2
:0636C3001583E038F0223F
:00000001FF
